:020000040800F2
:10000000700C0020A108000837020008390200081F
:100010003D020008410200084502000800000000FF
:10002000000000000000000000000000B30800080D
:100030004902000800000000B7080008B9080008DD
:10004000BB080008BB080008BB080008BB08000884
:10005000BB080008BB080008BB080008BB08000874
:10006000BB080008BB080008BB080008BB08000864
:10007000BB080008BB080008BB080008BB08000854
:10008000BB080008BB080008BB080008BB08000844
:10009000BB080008BB080008BB080008BB08000834
:1000A000BB080008BB080008BB080008BB08000824
:1000B000BB080008BB080008BB080008BB08000814
:1000C000BB080008BB080008BB080008BB08000804
:1000D000BB080008BB080008BB080008BB080008F4
:1000E000BB080008BB080008BB080008BB080008E4
:1000F000BB080008BB080008BB080008BB080008D4
:10010000BB080008BB080008BB080008BB080008C3
:10011000BB080008BB080008BB080008BB080008B3
:10012000BB080008BB080008BB080008BB080008A3
:10013000BB080008BB080008BB080008BB08000893
:10014000BB080008BB080008BB080008BB08000883
:10015000BB080008BB080008BB080008BB08000873
:10016000BB080008BB080008BB080008BB08000863
:10017000BB080008BB080008BB080008BB08000853
:10018000BB080008BB08000800F002F800F044F8C3
:100190000AA090E8000C82448344AAF10107DA45E2
:1001A00001D100F039F8AFF2090EBAE80F0013F0F0
:1001B000010F18BFFB1A43F0010318471824000071
:1001C00038240000103A24BF78C878C1FAD8520702
:1001D00024BF30C830C144BF04680C6070470000C1
:1001E0000023002400250026103A28BF78C1FBD840
:1001F000520728BF30C148BF0B607047782901F013
:100200005787732902F02F81002070471FB502F035
:10021000BEF91FBD10B510BD02F080F91146FFF701
:10022000F5FF00F08AF902F09EF903B4FFF7F2FF40
:1002300003BC01F0C8FA704700BFFEE700BFFEE74D
:1002400000BFFEE700BFFEE7704700009C48006863
:1002500040F080509A4908609A48006840F4404055
:1002600098490860964838380068954938390860D8
:100270000846006808600846006840F4805008603E
:100280009148091F0860081F006840F08070091F2E
:10029000086000BF8A484038006800F000700028FD
:1002A000F8D040F202708949086085483838006803
:1002B00020F003008249383908600846006840F0A1
:1002C0000200086000BF7E483838006800F00C006B
:1002D0000828F8D1704710B57D48006840F47000D8
:1002E0007B49086076484038006840F00100744956
:1002F0004039086000207249383908607048403839
:100300000068744908406E49403908607248091D08
:100310000860081F006820F48020091F0860002082
:10032000674934390860FFF791FF10BD70B50020B0
:100330000021022200230224614D383D2D6805F082
:100340000C0020B1042806D0082829D107E0634D0D
:10035000634E356028E0634D614E356024E0584DB2
:100360003C3D2D68C5F38053554D3C3D2D6805F04F
:100370003F044BB9594DB5FBF4F5514E3C3E366840
:10038000C6F3881605FB06F14D4D3C3D2D68C5F3BF
:1003900001456D1C6A00B1FBF2F5514E356003E07A
:1003A0004E4D4F4E356000BF00BF454D383D2D6866
:1003B000C5F303154C4E705D494D2D68C540484E40
:1003C000356070BD01466FF07F424FF0E0235A6107
:1003D00000229A6105221A6111E000224FF0E02309
:1003E0009A613F4A12684FF47A73B2FBF3F2C2F19A
:1003F000807000BF4FF0E02292698242FAD80A1E54
:10040000A1F10101E9D14FF0E022126922F00102CD
:100410004FF0E0231A61704701466FF07F424FF0C2
:10042000E0235A6100229A6105221A6111E000223C
:100430004FF0E0239A612A4A126842F21073B2FB2D
:10044000F3F2C2F1807000BF4FF0E0229269824265
:10045000FAD80A1EA1F10101E9D14FF0E022126998
:1004600022F001024FF0E0231A61704701466FF05D
:100470007F424FF0E0235A6100229A6105221A61FF
:1004800010E000224FF0E0239A61154A1268174BE2
:10049000B2FBF3F2C2F1807000BF4FF0E02292692C
:1004A0008242FAD80A1EA1F10101EAD14FF0E022FE
:1004B000126922F001024FF0E0231A617047000038
:1004C000403802400070004010640107003C0240C8
:1004D00088ED00E0FFFFF6FE103000240024F40059
:1004E0000000002000127A0004000020A086010015
:1004F0000FB410B5044614B1032C19D10FE02CA091
:1005000001F07AFD982203A92E4801F0E9FE2D4959
:1005100015312DA001F070FD01F09DF909E02FA02B
:1005200001F06AFD01F097F900203149087000E000
:1005300000BF00BF10BC5DF814FB4FF000602D49F8
:10054000086007230222C821102000F01EF94FF492
:10055000407000F0C5F900214FF4E13001F0D4F80B
:10056000AFF27301002001F045F901F074F90024A5
:1005700021A001F041FD1AE01D48007890B9204605
:10058000641C64280ED3002401201949087005203A
:100590001D4908731DA11C480D3001F07DFE1A484D
:1005A00001F043F90A2001F01FF901F07FF9E3E7B8
:1005B00052585F5354415F534543434553530D0ACB
:1005C000000000004C000020726620676574205017
:1005D00061636B65743A25730D0A000054585F53CC
:1005E00054415F534543434553530D0A00000000F7
:1005F0001400002008ED00E048656C6C6F20576F18
:10060000726C64210D0A0000E400002068656C6CC7
:100610006F0000001CB500200190009000F01AFB54
:100620009948006840F480309749086000BF9648B8
:10063000006800F4003000900198401C0190009880
:1006400018B90198B0F5A04FF1D18F48006800F4B7
:10065000003010B10120009001E0002000900098CF
:10066000012846D188484030006840F080508649D3
:10067000403108608548006840F440408349086084
:1006800081480830006880490831086008460068E1
:1006900040F4004008600846006840F4A05008603C
:1006A0007B48091F0860081F006840F08070091F20
:1006B000086000BF7448006800F000700028F9D09E
:1006C00040F20570734908606F480830006820F0F8
:1006D00003006D49083108600846006840F00200D8
:1006E000086000BF68480830006800F00C00082867
:1006F000F8D11CBD2DE9F84304460D4616461F46A9
:100700004FF0000800F0A6FA012000F0CCFA00F04B
:10071000EFFA8046B8F1010F35D15B4840300068F0
:1007200040F080505849403108605848006840F413
:10073000404056490860002000F078FB4FF4A0507C
:1007400000F07EFB4FF4805000F084FB33462A46D5
:1007500021464FF48000009700F00DFB012000F0CF
:100760001AFB00BF392000F0A5FA0028FAD040F2A9
:10077000057048490860022000F048FB00BF00F007
:100780004FFB0828FBD1BDE8F8832DE9FC41044666
:100790000D4616461F460020019000F05BFA01202E
:1007A00000F0CCFA3848006800F00200019001988F
:1007B000022834D134484030006840F0805032493B
:1007C000403108603148006840F440402F490860DB
:1007D000002000F02BFB4FF4A05000F031FB4FF451
:1007E000805000F037FB33462A4621460020009710
:1007F00000F0C1FA012000F0CEFA00BF392000F06D
:1008000059FA0028FAD040F2057022490860022007
:1008100000F0FCFA00BF00F003FB0828FBD1BDE8A4
:10082000FC811CB50121084600F0F0FB4FF48070FC
:10083000009002208DF8040000208DF806000120B1
:100840008DF8070003208DF805006946124800F076
:100850003DF91CBD1CB50121042000F0D7FB4FF46D
:100860000070009002208DF8040000208DF8060032
:1008700001208DF8070003208DF805006946074820
:1008800000F024F91CBD0000003802400070004058
:1008900019544007003C024000000240000802409A
:1008A0000948804709480047FEE7FEE7FEE7FEE704
:1008B000FEE7FEE7FEE7FEE7FEE7FEE70448054940
:1008C000054A064B70470000D7020008890100085E
:1008D00070020020700C00207004002070040020C2
:1008E00032490143324A1160704770B5002100233C
:1008F0000F22C4781CB32E4C246804F4E064C4F5C1
:10090000E064C4F30721C1F10404E3B20A4144786E
:100910009C40E1B28478144021430C07210E254C01
:1009200005786155047804F01F050124AC40057872
:100930006D11AD0005F1E025C5F8004109E004782E
:1009400004F01F050124AC401B4D0678761145F8D4
:10095000264070BD194A0A400243154B1B1F1A60FE
:10096000704739B1124A121D12680243104B1B1D09
:100970001A6006E00E4A121D126882430C4B1B1DC2
:100980001A607047042808D14FF0E021096941F04E
:1009900004014FF0E022116107E04FF0E021096906
:1009A00021F004014FF0E022116170470000FA05C8
:1009B0000CED00E000E400E080E100E080FFFF1FBC
:1009C00010B504469848844208D10121084600F039
:1009D00088FB0021012000F084FB76E093488442EC
:1009E00008D10121022000F07CFB0021022000F050
:1009F00078FB6AE08E48844208D10121042000F08F
:100A000070FB0021042000F06CFB5EE0894884420A
:100A100008D10121082000F064FB0021082000F02B
:100A200060FB52E08448844208D10121102000F08C
:100A300058FB0021102000F054FB46E07F48844220
:100A400008D10121202000F04CFB0021202000F0E3
:100A500048FB3AE07A48844208D10121402000F066
:100A600040FB0021402000F03CFB2EE07548844212
:100A700008D10121802000F034FB0021802000F00B
:100A800030FB22E07048844208D10121801500F03B
:100A900028FB0021A01500F024FB16E06B488442DF
:100AA00008D10121401500F01CFB0021601500F069
:100AB00018FB0AE06648844207D10121001500F0C6
:100AC00010FB0021201500F00CFB10BDF0B50A460C
:100AD00000210023002400BF3DE0012505FA01F3B9
:100AE000156805EA03049C4234D105684F000326CB
:100AF000BE40B543056015794E00B54006683543E4
:100B000005601579012D02D01579022D16D1856861
:100B10004F000326BE40B543856055794E00B54071
:100B2000866835438560456801268E40B54345603B
:100B3000456896798E40B6B235434560C5684F002A
:100B40000326BE40B543C560D5794E00B540C668A2
:100B50003543C560491C1029BFD3F0BD4FF6FF7166
:100B600001600021017141718171C171704708B547
:100B70004FF480320092009A0A430092009AC261B8
:100B8000C161009AC261C2690092C269009208BD47
:100B90000246002013690B400BB1012000E0002049
:100BA00070470146086980B27047024600205369C9
:100BB0000B400BB1012000E000207047014648695E
:100BC00080B2704701837047418370470AB1018347
:100BD00000E0418370474161704742694A40426189
:100BE0007047F0B5002300244D07ED0E02FA05F31F
:100BF000CE1000F1200555F826504E07F70E0F26AF
:100C0000BE40B543CF1000F1200646F82750CE1065
:100C100000F1200555F8265045EA0304CE1000F1F6
:100C2000200545F82640F0BD0000024000040240C7
:100C300000080240000C0240001002400014024074
:100C400000180240001C0240002002400024024024
:100C500000280240FA48006840F00100F8490860A6
:100C60000020F74908310860F5480068F549084058
:100C7000F3490860F448091D0860F448F0498431DC
:100C80000860F1481038091D0860ED48006820F43C
:100C90008020EB4908600020E9490C310860E849F0
:100CA0008C31086070470021E54A921C1170114692
:100CB0000870704710B501460022002300204A1139
:100CC000012A02D1DE4C236808E0022A03D1DC4C61
:100CD0007034236802E0DA4C7434236801F01F0298
:100CE000012494401C400CB1012000E0002010BD04
:100CF00038B5002000900024002500BF3120FFF708
:100D0000D9FF05460098401C00900098B0F5A04F10
:100D100001D0002DF2D03120FFF7CCFF08B1012423
:100D200000E00024204638BD01460020C44A106877
:100D300020F0F80040EAC10010607047C449086024
:100D400070470021BE4A703211701170012802D024
:100D500004280AD104E00121B94A7032117005E07B
:100D60000521B74A7032117000E000BF00BF704724
:100D7000B8490860704770B5049C41EA82150126A5
:100D8000C6EB530645EA0645054345EA0465AC4E05
:100D9000361D356070BDAE490866704710B58301D9
:100DA00043EA01731343A64C8434236010BDA84961
:100DB0008866704710B5830143EA016343EA027312
:100DC0009F4C8834236010BDA14908677047A04933
:100DD000C864704702460020994B0833186820F019
:100DE000EC6042EA01031843954B083318607047E2
:100DF00002460020924B0833186820F0784042EAFF
:100E0000010318438E4B08331860704701460020D9
:100E10008B4A0832106820F00300084310607047C6
:100E200087480830006800F00C0070470146002039
:100E3000834A0832106820F0F000084310607047C1
:100E4000014600207E4A0832106820F4E050084332
:100E50001060704701460020794A0832106820F47B
:100E6000604040EAC10010607047F0B500210022E8
:100E70000024022500260223714F08373F6807F03F
:100E80000C0121B1042905D0082937D105E0724FA2
:100E9000076036E0714F076033E0694F3F1D3F68E0
:100EA000C7F38056664F3F1D3F6807F03F036EB1A2
:100EB0006A4FB7FBF3F7DFF888C10CF1040CDCF8DC
:100EC00000C0CCF3881C07FB0CF40CE0624FB7FBAE
:100ED000F3F7DFF86CC10CF1040CDCF800C0CCF3C4
:100EE000881C07FB0CF4564F3F1D3F68C7F30147B2
:100EF0007F1C7D00B4FBF5F7076002E0564F0760EA
:100F000000BF00BF4E4F08373F6807F0F0010909E6
:100F1000534F7A5C0768D7404760494F08373F68AE
:100F200007F4E051890A4E4F7A5C4768D7408760E2
:100F3000434F08373F6807F46041490B484F7A5CDC
:100F40004768D740C760F0BD002100F44072B2F599
:100F5000407F0AD13A4A0832116821F4F811414A17
:100F600002401143364A08321160354A7032126825
:100F7000C0F30B031A43324B70331A607047354984
:100F80004439086070473349403908607047364932
:100F90000860704701460020294A8C32106820F012
:100FA0001F004A1E1043264A8C32106070470146CB
:100FB0000020234A8C32106820F4F8504A1E40EA80
:100FC00002201F4A8C3210607047014600201C4AE4
:100FD0008C32106820F440100843106070470146BE
:100FE0000020174A8C32106820F44000084310603B
:100FF000704701460020124A8C32106820F44030BD
:1010000008431060704719490860704739B10C4AAD
:101010003032126802430A4B30331A6006E0084A45
:10102000303212688243064B30331A607047F9B190
:10103000034A343212680243014B34331A601CE015
:1010400000380240FFFFF6EA103000240030002094
:1010500000004742800E47420024F40000127A004C
:1010600015000020FFFCFF0F5C014742E0114742E2
:101070008F4A126882438E4B1A60704739B18C4A8E
:10108000121D126802438A4B1B1D1A6006E0884A33
:10109000121D12688243864B1B1D1A60704739B1BE
:1010A000834A0C3212680243814B0C331A6006E00B
:1010B0007F4A0C32126882437D4B0C331A607047B2
:1010C00039B17B4A103212680243794B10331A60EF
:1010D00006E0774A103212688243754B10331A606B
:1010E000704739B1724A243A12680243704B243B6C
:1010F0001A6006E06E4A243A126882436C4B243B25
:101100001A60704739B16A4A203A12680243684B44
:10111000203B1A6006E0664A203A12688243644B1C
:10112000203B1A60704739B1614A1C3A1268024389
:101130005F4B1C3B1A6006E05D4A1C3A1268824312
:101140005B4B1C3B1A60704739B1594A143A12681C
:101150000243574B143B1A6006E0554A143A126892
:101160008243534B143B1A60704739B1504A103ACE
:10117000126802434E4B103B1A6006E04C4A103A8C
:10118000126882434A4B103B1A60704739B1484A93
:101190001C3212680243464B1C331A6006E0444A74
:1011A0001C3212688243424B1C331A60704739B1BB
:1011B0003F4A2032126802433D4B20331A6006E05A
:1011C0003B4A203212688243394B20331A60704701
:1011D00039B1374A243212680243354B24331A603E
:1011E00006E0334A243212688243314B24331A60BA
:1011F000704739B12E4A2C32126802432C4B2C33E3
:101200001A6006E02A4A2C3212688243284B2C339B
:101210001A60704739B1264A303212680243244BB3
:1012200030331A6006E0224A303212688243204B83
:1012300030331A607047012808D11D493C310968D4
:1012400041F008011A4A3C32116007E018493C316C
:10125000096821F00801164A3C321160704739B123
:10126000134A273A12780243114B273B1A7006E0C3
:101270000F4A273A127882430D4B273B1A7070476A
:101280000B484030006840F08070094940310860E8
:10129000704701460020064A283A12680A400AB1FF
:1012A000012000E00020704701492639087070478E
:1012B0003438024010B50446FA48844208D101216E
:1012C0001020FFF752FF00211020FFF74EFF57E0DC
:1012D000F548844209D101214804FFF735FF002178
:1012E0004FF40030FFF730FF4AE0F048844209D164
:1012F00001218804FFF728FF00214FF48020FFF729
:1013000023FF3DE0EA48844209D10121C804FFF7E8
:101310001BFF00214FF40020FFF716FF30E0E548E7
:10132000844209D101210805FFF70EFF00214FF487
:101330008010FFF709FF23E0DF48844208D1012134
:101340002020FFF712FF00212020FFF70EFF17E0FB
:10135000DA48844209D101218807FFF7F5FE002110
:101360004FF08040FFF7F0FE0AE0D548844207D1F5
:1013700001214005FFF7E8FE00216005FFF7E4FECC
:1013800010BD2DE9FF4705460E460024A14600BFCB
:10139000A046B08900B100BF2C8A24F44054F088E4
:1013A00004432C82AC8941F20C608443B0883189BB
:1013B0000843718908430443AC81AC8A24F4407427
:1013C000B0890443AC826846FFF74FFDB5488542BB
:1013D00002D0B948854202D1DDF80C9001E0DDF879
:1013E0000890A88900F4004040B109EBC90000EB67
:1013F000091031684900B0FBF1F707E009EBC900BB
:1014000000EB091031688900B0FBF1F76420B7FBED
:10141000F0F004012009642101FB1078A88900F490
:10142000004040B1322000EBC800B0FBF1F000F00A
:101430000700044308E0322000EB08106421B0FBF1
:10144000F1F000F00F0004432C81BDE8FF874FF45A
:101450001651016000218180C18001810C214181F0
:1014600000218181704710B502460020108A20F4C7
:1014700070600B884C8823438C882343CC8823439B
:101480001843108210BD0021018041808180C180FD
:10149000704721B1828942F40052828104E082893E
:1014A0004DF6FF731A4082817047028B02F47F422F
:1014B0000283028B0A430283704721B1828942F47E
:1014C0000042828103E08289C2F30E02828170476A
:1014D00021B1828A42F40062828204E0828A4FF261
:1014E000FF731A4082827047C1F3080282807047FE
:1014F00001468888C0F308007047028A4FF6F073EF
:101500001A400282028A0A430282704721B182890C
:1015100042F00202828104E082894FF6FD731A4094
:101520008281704782894FF2FF731A4082818289DB
:101530000A4382817047028A4FF6DF731A400282A3
:10154000028A0A430282704721B1028A42F4804231
:10155000028204E0028A4BF6FF731A40028270474F
:10156000818941F001018181704721B1828A42F075
:101570000802828204E0828A4FF6F7731A40828260
:101580007047028BD2B20283028B42EA01220283AD
:10159000704721B1828A42F02002828204E0828A6E
:1015A0004FF6DF731A408282704721B1828A42F07F
:1015B0001002828204E0828A4FF6EF731A40828220
:1015C0007047828A4FF6FB731A408282828A0A43EE
:1015D0008282704721B1828A42F00202828204E054
:1015E000828A4FF6FD731A40828270471AB1838A4D
:1015F0000B43838202E0838A8B4383827047F0B57A
:101600000346002400260025002040F66A17B94250
:1016100000D100BF1846C1F3421401F01F06012794
:1016200007FA06F5012C01D10C3004E0022C01D19F
:10163000103000E014301AB107682F43076002E051
:101640000768AF430760F0BD02460020B1F5007F98
:1016500000D100BF13880B400BB1012000E0002037
:10166000704701F40072B2F5007F00D100BFCA4399
:101670000280704770B50246002400230025002038
:1016800040F66A16B14200D100BFC1F3421501F025
:101690001F03012606FA03F3012D13D19689334067
:1016A00017E00000001001400044004000480040E6
:1016B000004C004000500040001401400078004001
:1016C000007C0040022D02D1168A334001E0968A48
:1016D00033400C12012606FA04F41688344013B184
:1016E0000CB1012000E0002070BD10B500220023E5
:1016F00040F66A14A14200D100BF0A1201249440AE
:10170000A3B2DC43048010BD30B587B004460D465B
:1017100001210846FFF77AFC01211020FFF7D0FCD9
:10172000072209212E48FFF75CFA07220A212C48DC
:10173000FFF757FA05A8FFF711FA4FF4C0600590BC
:1017400002208DF8190000208DF81A0002208DF873
:10175000180001208DF81B0005A92148FFF7B6F9F4
:1017600001940020ADF80800ADF80A00ADF80C00B7
:10177000ADF810000C20ADF80E0001A91948FFF7D4
:1017800000FE01211748FFF784FE07B030BD10B5F9
:10179000044600BF40211348FFF756FF0028F9D048
:1017A00021461048FFF7A0FE10BD70B504460D4657
:1017B00003E02078FFF7EBFF641C281EA5F1010170
:1017C0008DB2F6D170BD00BF704700BF054A1288C8
:1017D00002F04002002AF9D0C2B2024B9A80704750
:1017E000000002400010014010B504462046FEF7FC
:1017F000E9FD10BD70B505460C464FF47A70FFF751
:10180000F3FF00F066FB6B48007800F0F6F9642007
:10181000FFF7EAFF0CB16848046070BD10B5002006
:101820006649087000F07FFA10BD10B504466348A1
:101830000078012801D000F059F901205F490870B3
:1018400004F10D015EA000F0D7FB082104F10D00AA
:1018500000F080F910BD10B502205849087000F062
:101860004DF95BA000F0C8FB10BD70477047704792
:101870005048007840B270474E4A1070704770B5BB
:1018800004460D4614B1012C0DD108E003204B494C
:10189000087048480178002000F04BFA04E004206A
:1018A0004649087000E000BF00BF70BD30B5A3B06E
:1018B00042480078032801DB23B030BD3F48007860
:1018C00000B9F9E700F028F904460CB1FF2C00D16B
:1018D000F2E73A480278214641A000F08DFB04F07F
:1018E0002000B0B144A000F087FB00F022F900F026
:1018F0001AF90020314908708C224249684600F0EC
:10190000EFFC40480C380EC803202B4D2D68A8472B
:101910004EE004F01000B0B13BA000F06DFB0020E1
:101920002649087000F005F900F0FDF88C223549D1
:10193000684600F0D5FC33480C380EC803201E4D15
:101940002D68A84734E004F0400020B332A000F036
:1019500053FB80212B48093000F0F4FC0822294970
:101960000931612000F09FF800F0E3F800F0DBF8A7
:1019700000201249087010480068C8B18C22214923
:10198000684600F0ADFC1F480C380EC800200A4D18
:101990002D68A8470CE004F0600048B121A000F0D9
:1019A0002BFB00200549087000F0C3F800F0BBF8DD
:1019B00000BF81E7390000203400002038000020FB
:1019C00073656E6420646174613A25730A000000D7
:1019D000656E74657220746F20726563760A00000C
:1019E0007374617475733A2578202072664D6F6444
:1019F000653A25780A00000054585F44535F464C0E
:101A000041470A00800100204D41585F52545F4613
:101A10004C41470A0000000052585F44525F464C58
:101A200041470A0052585F54585F464C41470A00EC
:101A300010B504462046FEF719FD10BD70B50546E9
:101A40000C4600F03FFA284600F08DFA204600F0E0
:101A50008AFA00F030FA70BD70B5044600F032FA30
:101A6000204600F080FA00F0A3FA054600F023FAC1
:101A7000284670BD2DE9F04107460D46164600F098
:101A800021FA0024384600F06EFA00BF04E0285D19
:101A900000F069FA601CC4B2B442F8DB002400F024
:101AA0000AFABDE8F0812DE9F04107460D461646D9
:101AB00000F008FA384600F056FA002404E000F07E
:101AC00077FA2855601CC4B2B442F8DB00F0F3F991
:101AD000BDE8F08110B50021FD20FFF7AFFF10BD7C
:101AE00010B50021FC20FFF7A9FF10BD10B58E2115
:101AF0002020FFF7A3FFFFF7F3FF10BD10B5FFF79E
:101B0000EFFF8F212020FFF799FFFFF7E3FF4FF44E
:101B10007A70FFF78DFF10BD10B50720FFF79CFF0F
:101B200000F0700010BD10B570212720FFF786FF70
:101B300010BD10B50021E120FFF780FF0021E22059
:101B4000FFF77CFF10BD10B5044621462520FFF7A6
:101B500075FF10BD70B504460D46FFF7BBFF2A4662
:101B60002146A020FFF786FF4FF4FA60FFF760FFE1
:101B700070BD70B504460D46FFF7CEFF064606F071
:101B8000400008B9002070BD2A4621466120FFF7B9
:101B90008AFF0120F7E770B504460D46FFF7BCFF4A
:101BA00010281DD0202802D0602823D109E08A48BF
:101BB0000088401C88490880FFF7BBFFFFF7B3FF90
:101BC00019E02A4621466120FFF76DFF834800682F
:101BD000401C82490860FFF7ACFFFFF7A4FF0AE052
:101BE0007F480088401C7E490880FFF7A2FFFFF76E
:101BF0009AFF00E000BF00BF70BD30B58BB0044657
:101C000078A103C9CDE9090178A00068089078A1FE
:101C100003C9CDE9060178A00068059077A00068A7
:101C2000049020255A215320FFF708FFA5215320B7
:101C3000FFF704FF0021E120FFF700FF0021E22071
:101C4000FFF7FCFE70212720FFF7F8FE012122207C
:101C5000FFF7F4FE03212320FFF7F0FE00212520EB
:101C6000FFF7ECFE08213120FFF7E8FE052264496A
:101C70003020FFF7FFFE052261492A20FFF7FAFE18
:101C8000052209A93F20FFF7F5FE062206A93A2002
:101C9000FFF7F0FE012205A93920FFF7EBFE032232
:101CA00008A93E20FFF7E6FE032204A93B20FFF728
:101CB000E1FE00213C20FFF7C1FE21462620FFF770
:101CC000BDFE73215020FFF7B9FE00212420FFF74D
:101CD000B5FE00212120FFF7B1FE29463D20FFF788
:101CE000ADFE002002900390052202A91F20FFF7FD
:101CF000DAFE9DF80C009DF80B10CDE900109DF860
:101D00000A309DF809209DF808103EA000F074F9F3
:101D1000052209A902A800F093FA10B144A000F02E
:101D20006BF90BB030BD10B500212020FFF786FE07
:101D300010BD70B588B005460C462AA103C9CDE98F
:101D400006012AA0006805903EA103C9CDE9030160
:101D50003EA00068029029A00068019020265A2128
:101D60005320FFF76BFEA5215320FFF767FE314696
:101D70003D20FFF763FEFFF7B3FE4FF4FA70FFF765
:101D800057FE8E212020FFF759FE29462520FFF718
:101D900055FE21462620FFF751FE052206A93F20C9
:101DA000FFF768FE062203A93A20FFF763FE01222F
:101DB00002A93920FFF75EFE032205A93E20FFF7A6
:101DC00059FE032201A93B20FFF754FE4FF4FA709D
:101DD000FFF72EFE08B070BD480000204400002030
:101DE0004A0000200A6D679C46000000F6375D003F
:101DF0004521EF2C5A420000010000000BDF0200D9
:101E00003C000020525F42425F63616C5F6461741A
:101E1000613A202530327820253032782025303242
:101E200078202530327820253032780A00000000F2
:101E300042425F63616C5F64617461206572726FBE
:101E4000720A00004521EFAC5A500000E10000008A
:101E500010B5012208216648FEF7B8FE10BD10B586
:101E6000002208216248FEF7B1FE10BD10B5012224
:101E700010215F48FEF7AAFE10BD10B50022102108
:101E80005B48FEF7A3FE10BD1CB504461020009071
:101E90008DF8044000208DF8060003208DF8050021
:101EA00069465348FEF712FE1CBD10B5102150487C
:101EB000FEF76EFE10BD10B5012240214C48FEF722
:101EC00085FE10BD10B5002240214948FEF77EFE78
:101ED00010BD1CB501210220FFF798F810200090DA
:101EE00000208DF8040003208DF805006946404865
:101EF000FEF7ECFD0820009000208DF80600012080
:101F00008DF8040003208DF8050069463848FEF777
:101F1000DDFD4020009000208DF8060001208DF8A6
:101F2000040003208DF8050069463148FEF7CEFD18
:101F30004FF40070009001208DF8040000208DF80F
:101F4000060003208DF8050000208DF80700694683
:101F50002748FEF7BBFD4FF400712548FEF734FE1D
:101F6000FFF7A9FF1CBD70B50446012000F03DF845
:101F70000120FFF789FF00250FE0FFF770FF04F055
:101F8000800010B1FFF772FF01E0FFF776FFFFF767
:101F90005FFF6006040E681CC5B2082DEDDB002053
:101FA000FFF772FFFFF75BFF002000F01EF870BD27
:101FB00070B50024012000F018F800250CE0FFF7B0
:101FC0004EFF6006040EFFF743FFFFF76EFF08B1F8
:101FD000601CC4B2681CC5B2082DF0DBFFF73FFFE0
:101FE000002000F002F8204670BD80F31088704792
:101FF00000040240704700000FB4044910B503AA62
:10200000029800F035FA10BC5DF814FB3000002097
:1020100070B5044685690068C10601D5302600E028
:102020002026C00707D070BDD4E901213046904773
:10203000206A401C20626D1EF6D570BD70B5044646
:1020400085690078C00707D170BDD4E9012120203F
:102050009047206A401C20626D1EF6D570BD70B599
:102060000C460546012A05D02878800600D5EA6985
:10207000002302E0012305E05B1C934202D2E05CF6
:102080000028F9D1A869E618C01AA861286A18447E
:1020900028622846FFF7BCFF04E0D5E9012114F8C7
:1020A000010B9047B442F8D32846FFF7C7FF70BD35
:1020B00070B504460D4621461068AFF300802188B4
:1020C000090502D50F4A7A4402E00E4A7A440E32DC
:1020D000002104F1240305E000F00F060009965DDD
:1020E0005E54491C0028F7D120780023000704D54E
:1020F000702D02D009B1022311322046BDE8704094
:1021000000F046B9CE0400002DE9F05F8946044690
:102110004FF0000ADFF824B1FB44C0F820A02046AD
:10212000E168884700287DD0252806D0D4E9012120
:102130009047206A401C2062F1E700255F46204658
:10214000E16888472028064607DB312E05D2B819FA
:1021500010F8200C08B10543F1E7A80701D525F0D8
:102160000405C4F81CA00027C4F818A02A2E09D022
:10217000304600F005FA38B304EB8708303EC8F863
:10218000186019E059F8041B204604EB870291619E
:10219000E1688847012F064618D1E069002820DA57
:1021A00025F020051DE0D8F8180000EB800006EBB4
:1021B00040003038C8F818002046E16888470646D5
:1021C00000F0DEF90028EED1012F0AD02E2E08D122
:1021D0002046E16888477F1C0646022F45F020050F
:1021E000C4DBA069002803DA404245F00105A06184
:1021F000E80701D025F01005A6B1A6F14100192885
:1022000002D8203645F400654A463146204625600E
:102210004D46FDF7F3FF60B1012807D0ED1D25F015
:10222000070000E007E000F1080978E705F104097C
:1022300075E730467AE7206ABDE8F09FA404000005
:1022400040EA010310B59B070FD1042A0DD310C833
:1022500008C9121F9C42F8D020BA19BA884201D985
:10226000012010BD4FF0FF3010BD1AB1D30703D0CD
:10227000521C07E0002010BD10F8013B11F8014B83
:102280001B1B07D110F8013B11F8014B1B1B01D19F
:10229000921EF1D1184610BD40EA0103024630B546
:1022A0009B0710D14FF0013400E008C208C91D1B84
:1022B0009D4315EAC41FF8D013F0FF0102F8011B7B
:1022C0000DD01B0AF8E711F8013B002B02F8013B87
:1022D00005D011F8013B002B02F8013BF3D130BDD2
:1022E00010B5203AC0F00B80B1E81850203AA0E8B1
:1022F0001850B1E81850A0E81850BFF4F5AF5FEAE5
:10230000027C24BFB1E81850A0E8185044BF18C997
:1023100018C0BDE810405FEA827C24BF51F8043B3E
:1023200040F8043B08BF7047D20728BF31F8023B92
:1023300048BF11F8012B28BF20F8023B48BF00F826
:10234000012B70474FF000020429C0F0128010F0FA
:10235000030C00F0A180CCF1040CBCF1020F18BFFB
:1023600000F8012BA8BF20F8022BA1EB0C0100F014
:1023700093B85FEAC17C24BF00F8012B00F8012B61
:1023800048BF00F8012B704770477047704770478F
:102390002DE9F0470D4699469246044600F124087F
:1023A0000168880604D5E06921F01001216000E091
:1023B0000120A84201DD471B00E00027A1697A192E
:1023C00002EB0900081AA0612078C00602D420465A
:1023D000FFF71EFE002608E0D4E901211AF80600E6
:1023E0009047206A401C761C20624E45F4DB207822
:1023F000C0060AD52046FFF70BFE06E0D4E901210E
:1024000030209047206A401C2062381EA7F1010747
:10241000F4DC07E0D4E9012118F805009047206AB0
:10242000401C2062281EA5F10105F3DC2046FFF7C1
:1024300005FE2078000602D50220BDE8F0870120C5
:10244000FBE710B5436913B1AFF3008001E0FFF77C
:1024500006FE012010BD127800F124010A7000224E
:102460004A700122EDE711684FF0FF32E9E7000002
:10247000074B70B50D467B4400F039F804462846FA
:1024800000F048F810B14FF0FF3070BD204670BD2D
:1024900051F3FFFF4FF0000200B5134694469646F5
:1024A000203922BFA0E80C50A0E80C50B1F1200167
:1024B000BFF4F7AF090728BFA0E80C5048BF0CC015
:1024C0005DF804EB890028BF40F8042B08BF704773
:1024D00048BF20F8022B11F0804F18BF00F8012BE5
:1024E0007047000001694A1C02610878704700B516
:1024F0008FB0CDE901310021059105497944CDE93D
:10250000031011466846FFF7FFFD0FB000BD000045
:10251000E5FFFFFF007B00F080007047754600F08C
:102520002BF8AE4605006946534620F00700854665
:1025300018B020B5FEF7C2F9BDE820404FF0000604
:102540004FF000074FF000084FF0000B21F007019B
:10255000AC46ACE8C009ACE8C009ACE8C009ACE8DE
:10256000C0098D46704710B50446AFF30080204681
:10257000BDE81040FDF759BE004870470C0200202E
:1025800030380A2801D201207047002070474FF0F0
:102590004070E1EE100A704730313233343536374F
:1025A0003839414243444546403058003031323397
:1025B0003435363738396162636465664030780097
:1025C00004000008000000000000000200010000FC
:1025D00010000000F4250008000000204C0000005E
:1025E000C4010008402600084C000020240C000014
:1025F000E001000800E1F505000000000000000017
:10260000010203040607080901000000000102039B
:10261000040102030406070809000000000000008E
:102620000000000000000000000000000015000095
:10263000CCCCCCCCCC080000000000000000000096
:040000050800018965
:00000001FF
